:0200000480007A
:100000006F004005732F2034930F8000630AFF03B5
:10001000930F90006306FF03930FB0006302FF038A
:10002000170F0000130F0F2063040F0067000F006D
:10003000732F203463540F006F00400093E19153FD
:10004000171F000023203FFC171F0000232E0FFA6C
:100050006FF01FFF930000001301000093010000E8
:10006000130200009302000013030000930300003A
:100070001304000093040000130500009305000022
:10008000130600009306000013070000930700000A
:1000900013080000930800001309000093090000F2
:1000A000130A0000930A0000130B0000930B0000DA
:1000B000130C0000930C0000130D0000930D0000C2
:1000C000130E0000930E0000130F0000930F0000AA
:1000D000732540F16310050097020000938202012E
:1000E000739052307350447497020000938202015F
:1000F00073905230735000189702000093824202AE
:10010000739052309B021000939252039382F2FF3D
:100110007390023B9302F0017390023A73504030A7
:100120009702000093824201739052307350203046
:100130007350303093010000970200009382C2ECAC
:1001400073905230130510001315F501635C050020
:100150000F00F00F930110009308D0051305000065
:100160007300000093020000638A02007390521033
:10017000B7B200009B82921073902230735000300F
:10018000372500001B05058073200530970200000D
:100190009382420173901234732540F17300203032
:1001A00097030000938303059B02F0FF9392F203F1
:1001B000B3C27200930120001303100097040000E3
:1001C0009384040193030000E7830200930130004D
:1001D00013035000970400009384440193830400A8
:1001E000838302006F00C0006F0040026310300282
:1001F0000F00F00F638001009391110093E1110053
:100200009308D00513850100730000000F00F00F64
:10021000930110009308D00513050000730000003F
:10022000130520006388A100130530006384A1003A
:100230006FF01FFCE39E93FAF3232034E39A63FAF2
:100240007390143473002030731000C0000000005D
:10025000000000000000000000000000000000009E
:10026000000000000000000000000000000000008E
:10027000000000000000000000000000000000007E
:1010000000000000000000000000000000000000E0
:1010100000000000000000000000000000000000D0
:1010200000000000000000000000000000000000C0
:1010300000000000000000000000000000000000B0
:081040000000000000000000A8
:040000058000000077
:00000001FF
